ARM Linker, 4.1 [Build 713] [Standard]

==============================================================================

Section Cross References

    system_xn11lxxx.o(.text) refers to rt_memcpy.o(.emb_text) for __aeabi_memcpy4
    system_xn11lxxx.o(.text) refers to aeabi_sdiv.o(.text) for __aeabi_uidivmod
    system_xn11lxxx.o(.text) refers to system_xn11lxxx.o(.constdata) for .constdata
    system_xn11lxxx.o(.text) refers to system_xn11lxxx.o(.data) for MainClock
    startup_xn11lxxx.o(STACK) refers (Special) to heapauxi.o(.text) for __use_two_region_memory
    startup_xn11lxxx.o(HEAP) refers (Special) to heapauxi.o(.text) for __use_two_region_memory
    startup_xn11lxxx.o(RESET) refers (Special) to heapauxi.o(.text) for __use_two_region_memory
    startup_xn11lxxx.o(RESET) refers to startup_xn11lxxx.o(STACK) for __initial_sp
    startup_xn11lxxx.o(RESET) refers to startup_xn11lxxx.o(.text) for Reset_Handler
    startup_xn11lxxx.o(RESET) refers to xn_uart.o(.text) for UART0_IRQHandler
    startup_xn11lxxx.o(.text) refers (Special) to heapauxi.o(.text) for __use_two_region_memory
    startup_xn11lxxx.o(.text) refers to __main.o(!!!main) for __main
    startup_xn11lxxx.o(.text) refers to startup_xn11lxxx.o(HEAP) for Heap_Mem
    startup_xn11lxxx.o(.text) refers to startup_xn11lxxx.o(STACK) for Stack_Mem
    xn_uart.o(.text) refers to aeabi_sdiv.o(.text) for __aeabi_uidivmod
    xn_uart.o(.text) refers to system_xn11lxxx.o(.data) for MainClock
    xn_uart.o(.text) refers to xn_uart.o(.data) for UART0Head
    xn_uart.o(.text) refers to xn_uart.o(.bss) for UART0Buffer
    main.o(.text) refers to system_xn11lxxx.o(.text) for SystemCoreClockUpdate
    main.o(.text) refers to xn_uart.o(.text) for SetUART0Pin
    rt_memcpy.o(.text) refers to rt_memcpy.o(.emb_text) for __aeabi_memcpy4
    __main.o(!!!main) refers to rtentry.o(.ARM.Collect$$rtentry$$00000000) for __rt_entry
    rtentry.o(.ARM.Collect$$rtentry$$00000000) refers (Special) to rtentry2.o(.ARM.Collect$$rtentry$$0000000A) for __rt_entry_li
    rtentry.o(.ARM.Collect$$rtentry$$00000000) refers (Special) to rtentry2.o(.ARM.Collect$$rtentry$$0000000D) for __rt_entry_main
    rtentry.o(.ARM.Collect$$rtentry$$00000000) refers (Special) to rtentry2.o(.ARM.Collect$$rtentry$$0000000C) for __rt_entry_postli_1
    rtentry.o(.ARM.Collect$$rtentry$$00000000) refers (Special) to rtentry2.o(.ARM.Collect$$rtentry$$00000009) for __rt_entry_postsh_1
    rtentry.o(.ARM.Collect$$rtentry$$00000000) refers (Special) to rtentry2.o(.ARM.Collect$$rtentry$$00000002) for __rt_entry_presh_1
    rtentry.o(.ARM.Collect$$rtentry$$00000000) refers (Special) to rtentry4.o(.ARM.Collect$$rtentry$$00000004) for __rt_entry_sh
    rtentry.o(.ARM.exidx) refers (Special) to rtentry2.o(.ARM.Collect$$rtentry$$0000000A) for __rt_entry_li
    rtentry.o(.ARM.exidx) refers (Special) to rtentry2.o(.ARM.Collect$$rtentry$$0000000D) for __rt_entry_main
    rtentry.o(.ARM.exidx) refers (Special) to rtentry2.o(.ARM.Collect$$rtentry$$0000000C) for __rt_entry_postli_1
    rtentry.o(.ARM.exidx) refers (Special) to rtentry2.o(.ARM.Collect$$rtentry$$00000009) for __rt_entry_postsh_1
    rtentry.o(.ARM.exidx) refers (Special) to rtentry2.o(.ARM.Collect$$rtentry$$00000002) for __rt_entry_presh_1
    rtentry.o(.ARM.exidx) refers (Special) to rtentry4.o(.ARM.Collect$$rtentry$$00000004) for __rt_entry_sh
    rtentry.o(.ARM.exidx) refers to rtentry.o(.ARM.Collect$$rtentry$$00000000) for .ARM.Collect$$rtentry$$00000000
    aeabi_idiv0_sigfpe.o(.text) refers to rt_div0.o(.text) for __rt_div0
    rtentry2.o(.ARM.Collect$$rtentry$$00000008) refers to boardinit2.o(.text) for _platform_post_stackheap_init
    rtentry2.o(.ARM.Collect$$rtentry$$0000000A) refers to libinit.o(.ARM.Collect$$libinit$$00000000) for __rt_lib_init
    rtentry2.o(.ARM.Collect$$rtentry$$0000000B) refers to boardinit3.o(.text) for _platform_post_lib_init
    rtentry2.o(.ARM.Collect$$rtentry$$0000000D) refers to main.o(.text) for main
    rtentry2.o(.ARM.Collect$$rtentry$$0000000D) refers to exit.o(.text) for exit
    rtentry2.o(.ARM.exidx) refers to rtentry2.o(.ARM.Collect$$rtentry$$00000001) for .ARM.Collect$$rtentry$$00000001
    rtentry2.o(.ARM.exidx) refers to rtentry2.o(.ARM.Collect$$rtentry$$00000002) for .ARM.Collect$$rtentry$$00000002
    rtentry2.o(.ARM.exidx) refers to rtentry2.o(.ARM.Collect$$rtentry$$00000008) for .ARM.Collect$$rtentry$$00000008
    rtentry2.o(.ARM.exidx) refers to rtentry2.o(.ARM.Collect$$rtentry$$00000009) for .ARM.Collect$$rtentry$$00000009
    rtentry2.o(.ARM.exidx) refers to rtentry2.o(.ARM.Collect$$rtentry$$0000000A) for .ARM.Collect$$rtentry$$0000000A
    rtentry2.o(.ARM.exidx) refers to rtentry2.o(.ARM.Collect$$rtentry$$0000000B) for .ARM.Collect$$rtentry$$0000000B
    rtentry2.o(.ARM.exidx) refers to rtentry2.o(.ARM.Collect$$rtentry$$0000000C) for .ARM.Collect$$rtentry$$0000000C
    rtentry2.o(.ARM.exidx) refers to rtentry2.o(.ARM.Collect$$rtentry$$0000000D) for .ARM.Collect$$rtentry$$0000000D
    rtentry4.o(.ARM.Collect$$rtentry$$00000004) refers to sys_stackheap_outer.o(.text) for __user_setup_stackheap
    rtentry4.o(.ARM.exidx) refers to rtentry4.o(.ARM.Collect$$rtentry$$00000004) for .ARM.Collect$$rtentry$$00000004
    rt_div0.o(.text) refers to defsig_fpe_outer.o(.text) for __rt_SIGFPE
    sys_stackheap_outer.o(.text) refers to libspace.o(.text) for __user_perproc_libspace
    sys_stackheap_outer.o(.text) refers to startup_xn11lxxx.o(.text) for __user_initial_stackheap
    sys_stackheap_outer.o(__vectab_stack_and_reset_area) refers to tempstk.o(.text) for __temporary_stack_top
    sys_stackheap_outer.o(__vectab_stack_and_reset_area) refers to __main.o(!!!main) for __main
    exit.o(.text) refers to rtexit.o(.ARM.Collect$$rtexit$$00000000) for __rt_exit
    defsig_fpe_outer.o(.text) refers to defsig_fpe_inner.o(.text) for __rt_SIGFPE_inner
    defsig_fpe_outer.o(.text) refers to defsig_exit.o(.text) for __sig_exit
    defsig_fpe_formal.o(.text) refers to rt_raise.o(.text) for __rt_raise
    libinit.o(.ARM.Collect$$libinit$$00000000) refers (Special) to libinit2.o(.ARM.Collect$$libinit$$0000002A) for __rt_lib_init_alloca_1
    libinit.o(.ARM.Collect$$libinit$$00000000) refers (Special) to libinit2.o(.ARM.Collect$$libinit$$00000028) for __rt_lib_init_argv_1
    libinit.o(.ARM.Collect$$libinit$$00000000) refers (Special) to libinit2.o(.ARM.Collect$$libinit$$00000017) for __rt_lib_init_atexit_1
    libinit.o(.ARM.Collect$$libinit$$00000000) refers (Special) to libinit2.o(.ARM.Collect$$libinit$$0000001D) for __rt_lib_init_clock_1
    libinit.o(.ARM.Collect$$libinit$$00000000) refers (Special) to libinit2.o(.ARM.Collect$$libinit$$0000002E) for __rt_lib_init_cpp_1
    libinit.o(.ARM.Collect$$libinit$$00000000) refers (Special) to libinit2.o(.ARM.Collect$$libinit$$0000002C) for __rt_lib_init_exceptions_1
    libinit.o(.ARM.Collect$$libinit$$00000000) refers (Special) to libinit2.o(.ARM.Collect$$libinit$$0000001B) for __rt_lib_init_fp_trap_1
    libinit.o(.ARM.Collect$$libinit$$00000000) refers (Special) to libinit2.o(.ARM.Collect$$libinit$$0000001F) for __rt_lib_init_getenv_1
    libinit.o(.ARM.Collect$$libinit$$00000000) refers (Special) to libinit2.o(.ARM.Collect$$libinit$$00000006) for __rt_lib_init_heap_1
    libinit.o(.ARM.Collect$$libinit$$00000000) refers (Special) to libinit2.o(.ARM.Collect$$libinit$$0000000D) for __rt_lib_init_lc_collate_1
    libinit.o(.ARM.Collect$$libinit$$00000000) refers (Special) to libinit2.o(.ARM.Collect$$libinit$$0000000F) for __rt_lib_init_lc_ctype_1
    libinit.o(.ARM.Collect$$libinit$$00000000) refers (Special) to libinit2.o(.ARM.Collect$$libinit$$00000011) for __rt_lib_init_lc_monetary_1
    libinit.o(.ARM.Collect$$libinit$$00000000) refers (Special) to libinit2.o(.ARM.Collect$$libinit$$00000013) for __rt_lib_init_lc_numeric_1
    libinit.o(.ARM.Collect$$libinit$$00000000) refers (Special) to libinit2.o(.ARM.Collect$$libinit$$00000015) for __rt_lib_init_lc_time_1
    libinit.o(.ARM.Collect$$libinit$$00000000) refers (Special) to libinit2.o(.ARM.Collect$$libinit$$0000000A) for __rt_lib_init_rand_1
    libinit.o(.ARM.Collect$$libinit$$00000000) refers (Special) to libinit2.o(.ARM.Collect$$libinit$$0000002F) for __rt_lib_init_return
    libinit.o(.ARM.Collect$$libinit$$00000000) refers (Special) to libinit2.o(.ARM.Collect$$libinit$$00000019) for __rt_lib_init_signal_1
    libinit.o(.ARM.Collect$$libinit$$00000000) refers (Special) to libinit2.o(.ARM.Collect$$libinit$$00000021) for __rt_lib_init_stdio_1
    libinit.o(.ARM.Collect$$libinit$$00000000) refers (Special) to libinit2.o(.ARM.Collect$$libinit$$00000008) for __rt_lib_init_user_alloc_1
    libspace.o(.text) refers to libspace.o(.bss) for __libspace_start
    rtexit.o(.ARM.Collect$$rtexit$$00000000) refers (Special) to rtexit2.o(.ARM.Collect$$rtexit$$00000004) for __rt_exit_exit
    rtexit.o(.ARM.Collect$$rtexit$$00000000) refers (Special) to rtexit2.o(.ARM.Collect$$rtexit$$00000003) for __rt_exit_ls
    rtexit.o(.ARM.Collect$$rtexit$$00000000) refers (Special) to rtexit2.o(.ARM.Collect$$rtexit$$00000002) for __rt_exit_prels_1
    rtexit.o(.ARM.exidx) refers (Special) to rtexit2.o(.ARM.Collect$$rtexit$$00000004) for __rt_exit_exit
    rtexit.o(.ARM.exidx) refers (Special) to rtexit2.o(.ARM.Collect$$rtexit$$00000003) for __rt_exit_ls
    rtexit.o(.ARM.exidx) refers (Special) to rtexit2.o(.ARM.Collect$$rtexit$$00000002) for __rt_exit_prels_1
    rtexit.o(.ARM.exidx) refers to rtexit.o(.ARM.Collect$$rtexit$$00000000) for .ARM.Collect$$rtexit$$00000000
    rt_raise.o(.text) refers to __raise.o(.text) for __raise
    rt_raise.o(.text) refers to sys_exit.o(.text) for _sys_exit
    defsig_exit.o(.text) refers to sys_exit.o(.text) for _sys_exit
    defsig_fpe_inner.o(.text) refers to defsig_general.o(.text) for __default_signal_display
    libinit2.o(.ARM.Collect$$libinit$$0000000C) refers to libinit2.o(.ARM.Collect$$libinit$$0000000B) for .ARM.Collect$$libinit$$0000000B
    libinit2.o(.ARM.Collect$$libinit$$0000000E) refers to libinit2.o(.ARM.Collect$$libinit$$0000000B) for .ARM.Collect$$libinit$$0000000B
    libinit2.o(.ARM.Collect$$libinit$$00000010) refers to libinit2.o(.ARM.Collect$$libinit$$0000000B) for .ARM.Collect$$libinit$$0000000B
    libinit2.o(.ARM.Collect$$libinit$$00000012) refers to libinit2.o(.ARM.Collect$$libinit$$0000000B) for .ARM.Collect$$libinit$$0000000B
    libinit2.o(.ARM.Collect$$libinit$$00000014) refers to libinit2.o(.ARM.Collect$$libinit$$0000000B) for .ARM.Collect$$libinit$$0000000B
    libinit2.o(.ARM.Collect$$libinit$$00000022) refers to argv_veneer.o(.text) for __ARM_argv_veneer
    libinit2.o(.ARM.Collect$$libinit$$00000023) refers to argv_veneer.o(.text) for __ARM_argv_veneer
    sys_exit.o(.text) refers (Special) to use_no_semi.o(.text) for __I$use$semihosting
    sys_exit.o(.text) refers (Special) to indicate_semi.o(.text) for __semihosting_library_function
    rtexit2.o(.ARM.Collect$$rtexit$$00000003) refers to libshutdown.o(.ARM.Collect$$libshutdown$$00000000) for __rt_lib_shutdown
    rtexit2.o(.ARM.Collect$$rtexit$$00000004) refers to sys_exit.o(.text) for _sys_exit
    rtexit2.o(.ARM.exidx) refers to rtexit2.o(.ARM.Collect$$rtexit$$00000001) for .ARM.Collect$$rtexit$$00000001
    rtexit2.o(.ARM.exidx) refers to rtexit2.o(.ARM.Collect$$rtexit$$00000002) for .ARM.Collect$$rtexit$$00000002
    rtexit2.o(.ARM.exidx) refers to rtexit2.o(.ARM.Collect$$rtexit$$00000003) for .ARM.Collect$$rtexit$$00000003
    rtexit2.o(.ARM.exidx) refers to rtexit2.o(.ARM.Collect$$rtexit$$00000004) for .ARM.Collect$$rtexit$$00000004
    __raise.o(.text) refers to defsig.o(CL$$defsig) for __default_signal_handler
    defsig_general.o(.text) refers to sys_wrch.o(.text) for _ttywrch
    sys_wrch.o(.text) refers (Special) to use_no_semi.o(.text) for __I$use$semihosting
    sys_wrch.o(.text) refers (Special) to indicate_semi.o(.text) for __semihosting_library_function
    defsig.o(CL$$defsig) refers to defsig_fpe_inner.o(.text) for __rt_SIGFPE_inner
    defsig.o(CL$$defsig) refers to defsig_rtmem_inner.o(.text) for __rt_SIGRTMEM_inner
    _get_argv_nomalloc.o(.text) refers (Special) to hrguard.o(.text) for __heap_region$guard
    _get_argv_nomalloc.o(.text) refers to defsig_rtmem_outer.o(.text) for __rt_SIGRTMEM
    _get_argv_nomalloc.o(.text) refers to sys_command.o(.text) for _sys_command_string
    libshutdown.o(.ARM.Collect$$libshutdown$$00000000) refers (Special) to libshutdown2.o(.ARM.Collect$$libshutdown$$00000006) for __rt_lib_shutdown_fp_trap_1
    libshutdown.o(.ARM.Collect$$libshutdown$$00000000) refers (Special) to libshutdown2.o(.ARM.Collect$$libshutdown$$0000000E) for __rt_lib_shutdown_heap_1
    libshutdown.o(.ARM.Collect$$libshutdown$$00000000) refers (Special) to libshutdown2.o(.ARM.Collect$$libshutdown$$0000000F) for __rt_lib_shutdown_return
    libshutdown.o(.ARM.Collect$$libshutdown$$00000000) refers (Special) to libshutdown2.o(.ARM.Collect$$libshutdown$$00000009) for __rt_lib_shutdown_signal_1
    libshutdown.o(.ARM.Collect$$libshutdown$$00000000) refers (Special) to libshutdown2.o(.ARM.Collect$$libshutdown$$00000003) for __rt_lib_shutdown_stdio_1
    libshutdown.o(.ARM.Collect$$libshutdown$$00000000) refers (Special) to libshutdown2.o(.ARM.Collect$$libshutdown$$0000000B) for __rt_lib_shutdown_user_alloc_1
    sys_command.o(.text) refers (Special) to use_no_semi.o(.text) for __I$use$semihosting
    sys_command.o(.text) refers (Special) to indicate_semi.o(.text) for __semihosting_library_function
    defsig_abrt_inner.o(.text) refers to defsig_general.o(.text) for __default_signal_display
    defsig_rtred_inner.o(.text) refers to defsig_general.o(.text) for __default_signal_display
    defsig_rtmem_inner.o(.text) refers to defsig_general.o(.text) for __default_signal_display
    defsig_rtmem_outer.o(.text) refers to defsig_rtmem_inner.o(.text) for __rt_SIGRTMEM_inner
    defsig_rtmem_outer.o(.text) refers to defsig_exit.o(.text) for __sig_exit
    defsig_rtmem_formal.o(.text) refers to rt_raise.o(.text) for __rt_raise
    defsig_stak_inner.o(.text) refers to defsig_general.o(.text) for __default_signal_display
    defsig_pvfn_inner.o(.text) refers to defsig_general.o(.text) for __default_signal_display
    defsig_cppl_inner.o(.text) refers to defsig_general.o(.text) for __default_signal_display
    defsig_segv_inner.o(.text) refers to defsig_general.o(.text) for __default_signal_display
    defsig_other.o(.text) refers to defsig_general.o(.text) for __default_signal_display


==============================================================================

Removing Unused input sections from the image.

    Removing system_xn11lxxx.o(.emb_text), (8 bytes).
    Removing xn_uart.o(.emb_text), (8 bytes).
    Removing main.o(.emb_text), (8 bytes).

3 unused section(s) (total 24 bytes) removed from the image.

==============================================================================

Image Symbol Table

    Local Symbols

    Symbol Name                              Value     Ov Type        Size  Object(Section)

    ../../angel/boardlib.s                   0x00000000   Number         0  boardinit3.o ABSOLUTE
    ../../angel/boardlib.s                   0x00000000   Number         0  boardinit2.o ABSOLUTE
    ../../angel/boardlib.s                   0x00000000   Number         0  boardinit1.o ABSOLUTE
    ../../angel/boardlib.s                   0x00000000   Number         0  boardshut.o ABSOLUTE
    ../../angel/handlers.s                   0x00000000   Number         0  __scatter_zi.o ABSOLUTE
    ../../angel/handlers.s                   0x00000000   Number         0  __scatter_copy.o ABSOLUTE
    ../../angel/kernel.s                     0x00000000   Number         0  rtexit2.o ABSOLUTE
    ../../angel/kernel.s                     0x00000000   Number         0  rtentry4.o ABSOLUTE
    ../../angel/kernel.s                     0x00000000   Number         0  rtexit.o ABSOLUTE
    ../../angel/kernel.s                     0x00000000   Number         0  rtentry.o ABSOLUTE
    ../../angel/kernel.s                     0x00000000   Number         0  rtentry2.o ABSOLUTE
    ../../angel/rt.s                         0x00000000   Number         0  rt_div0.o ABSOLUTE
    ../../angel/rt.s                         0x00000000   Number         0  rt_raise.o ABSOLUTE
    ../../angel/rt.s                         0x00000000   Number         0  aeabi_idiv0.o ABSOLUTE
    ../../angel/rt.s                         0x00000000   Number         0  aeabi_idiv0_sigfpe.o ABSOLUTE
    ../../angel/scatterp.s                   0x00000000   Number         0  __scatter.o ABSOLUTE
    ../../angel/startup.s                    0x00000000   Number         0  __main.o ABSOLUTE
    ../../angel/sys.s                        0x00000000   Number         0  use_no_semi.o ABSOLUTE
    ../../angel/sys.s                        0x00000000   Number         0  tempstk.o ABSOLUTE
    ../../angel/sys.s                        0x00000000   Number         0  sys_stackheap_outer.o ABSOLUTE
    ../../angel/sys.s                        0x00000000   Number         0  libspace.o ABSOLUTE
    ../../angel/sys.s                        0x00000000   Number         0  indicate_semi.o ABSOLUTE
    ../../angel/sysapp.c                     0x00000000   Number         0  sys_wrch.o ABSOLUTE
    ../../angel/sysapp.c                     0x00000000   Number         0  sys_command.o ABSOLUTE
    ../../angel/sysapp.c                     0x00000000   Number         0  sys_exit.o ABSOLUTE
    ../../armsys.c                           0x00000000   Number         0  argv_veneer.o ABSOLUTE
    ../../armsys.c                           0x00000000   Number         0  _get_argv_nomalloc.o ABSOLUTE
    ../../armsys.c                           0x00000000   Number         0  no_argv.o ABSOLUTE
    ../../cfplib/fpinit.c                    0x00000000   Number         0  fpinit.o ABSOLUTE
    ../../division.s                         0x00000000   Number         0  aeabi_sdiv.o ABSOLUTE
    ../../division.s                         0x00000000   Number         0  aeabi_sdiv_div0.o ABSOLUTE
    ../../heapalloc.c                        0x00000000   Number         0  hrguard.o ABSOLUTE
    ../../heapaux.c                          0x00000000   Number         0  heapauxi.o ABSOLUTE
    ../../libinit.s                          0x00000000   Number         0  libinit.o ABSOLUTE
    ../../libinit.s                          0x00000000   Number         0  libshutdown2.o ABSOLUTE
    ../../libinit.s                          0x00000000   Number         0  libinit2.o ABSOLUTE
    ../../libinit.s                          0x00000000   Number         0  libshutdown.o ABSOLUTE
    ../../memcpset.c                         0x00000000   Number         0  rt_memcpy.o ABSOLUTE
    ../../memcpset.c                         0x00000000   Number         0  rt_memcpy.o ABSOLUTE
    ../../signal.c                           0x00000000   Number         0  defsig_stak_inner.o ABSOLUTE
    ../../signal.c                           0x00000000   Number         0  defsig_cppl_inner.o ABSOLUTE
    ../../signal.c                           0x00000000   Number         0  defsig_pvfn_inner.o ABSOLUTE
    ../../signal.c                           0x00000000   Number         0  defsig_segv_inner.o ABSOLUTE
    ../../signal.c                           0x00000000   Number         0  defsig_other.o ABSOLUTE
    ../../signal.c                           0x00000000   Number         0  defsig_exit.o ABSOLUTE
    ../../signal.c                           0x00000000   Number         0  defsig_general.o ABSOLUTE
    ../../signal.c                           0x00000000   Number         0  defsig_abrt_inner.o ABSOLUTE
    ../../signal.c                           0x00000000   Number         0  __raise.o ABSOLUTE
    ../../signal.c                           0x00000000   Number         0  defsig_rtred_inner.o ABSOLUTE
    ../../signal.c                           0x00000000   Number         0  defsig_fpe_inner.o ABSOLUTE
    ../../signal.c                           0x00000000   Number         0  defsig_fpe_outer.o ABSOLUTE
    ../../signal.c                           0x00000000   Number         0  defsig_fpe_formal.o ABSOLUTE
    ../../signal.c                           0x00000000   Number         0  defsig_rtmem_outer.o ABSOLUTE
    ../../signal.c                           0x00000000   Number         0  defsig_rtmem_inner.o ABSOLUTE
    ../../signal.c                           0x00000000   Number         0  defsig_rtmem_formal.o ABSOLUTE
    ../../signal.s                           0x00000000   Number         0  defsig.o ABSOLUTE
    ../../stdlib.c                           0x00000000   Number         0  exit.o ABSOLUTE
    ..\..\common\Core\CM0\CoreSupport\core_cm0.c 0x00000000   Number         0  core_cm0.o ABSOLUTE
    ..\..\common\Core\CM0\DeviceSupport\XN11L\startup\arm\startup_XN11Lxxx.s 0x00000000   Number         0  startup_xn11lxxx.o ABSOLUTE
    ..\..\common\Core\CM0\DeviceSupport\XN11L\system_XN11Lxxx.c 0x00000000   Number         0  system_xn11lxxx.o ABSOLUTE
    ..\..\common\Drivers\source\xn_uart.c    0x00000000   Number         0  xn_uart.o ABSOLUTE
    ..\\..\\common\\Core\\CM0\\DeviceSupport\\XN11L\\system_XN11Lxxx.c 0x00000000   Number         0  system_xn11lxxx.o ABSOLUTE
    ..\\..\\common\\Drivers\\source\\xn_uart.c 0x00000000   Number         0  xn_uart.o ABSOLUTE
    dc.s                                     0x00000000   Number         0  dc.o ABSOLUTE
    src\\main.c                              0x00000000   Number         0  main.o ABSOLUTE
    src\main.c                               0x00000000   Number         0  main.o ABSOLUTE
    RESET                                    0x10000000   Section      192  startup_xn11lxxx.o(RESET)
    !!!main                                  0x100000c0   Section        8  __main.o(!!!main)
    !!!scatter                               0x100000c8   Section       60  __scatter.o(!!!scatter)
    !!handler_copy                           0x10000104   Section       26  __scatter_copy.o(!!handler_copy)
    !!handler_zi                             0x10000120   Section       28  __scatter_zi.o(!!handler_zi)
    .ARM.Collect$$libinit$$00000000          0x1000013c   Section        6  libinit.o(.ARM.Collect$$libinit$$00000000)
    .ARM.Collect$$libinit$$00000006          0x10000142   Section        0  libinit2.o(.ARM.Collect$$libinit$$00000006)
    .ARM.Collect$$libinit$$00000008          0x10000142   Section        0  libinit2.o(.ARM.Collect$$libinit$$00000008)
    .ARM.Collect$$libinit$$0000000A          0x10000142   Section        0  libinit2.o(.ARM.Collect$$libinit$$0000000A)
    .ARM.Collect$$libinit$$0000000D          0x10000142   Section        0  libinit2.o(.ARM.Collect$$libinit$$0000000D)
    .ARM.Collect$$libinit$$0000000F          0x10000142   Section        0  libinit2.o(.ARM.Collect$$libinit$$0000000F)
    .ARM.Collect$$libinit$$00000011          0x10000142   Section        0  libinit2.o(.ARM.Collect$$libinit$$00000011)
    .ARM.Collect$$libinit$$00000013          0x10000142   Section        0  libinit2.o(.ARM.Collect$$libinit$$00000013)
    .ARM.Collect$$libinit$$00000015          0x10000142   Section        0  libinit2.o(.ARM.Collect$$libinit$$00000015)
    .ARM.Collect$$libinit$$00000017          0x10000142   Section        0  libinit2.o(.ARM.Collect$$libinit$$00000017)
    .ARM.Collect$$libinit$$00000019          0x10000142   Section        0  libinit2.o(.ARM.Collect$$libinit$$00000019)
    .ARM.Collect$$libinit$$0000001B          0x10000142   Section        0  libinit2.o(.ARM.Collect$$libinit$$0000001B)
    .ARM.Collect$$libinit$$0000001D          0x10000142   Section        0  libinit2.o(.ARM.Collect$$libinit$$0000001D)
    .ARM.Collect$$libinit$$0000001F          0x10000142   Section        0  libinit2.o(.ARM.Collect$$libinit$$0000001F)
    .ARM.Collect$$libinit$$00000021          0x10000142   Section        0  libinit2.o(.ARM.Collect$$libinit$$00000021)
    .ARM.Collect$$libinit$$00000028          0x10000142   Section        0  libinit2.o(.ARM.Collect$$libinit$$00000028)
    .ARM.Collect$$libinit$$0000002A          0x10000142   Section        0  libinit2.o(.ARM.Collect$$libinit$$0000002A)
    .ARM.Collect$$libinit$$0000002C          0x10000142   Section        0  libinit2.o(.ARM.Collect$$libinit$$0000002C)
    .ARM.Collect$$libinit$$0000002E          0x10000142   Section        0  libinit2.o(.ARM.Collect$$libinit$$0000002E)
    .ARM.Collect$$libinit$$0000002F          0x10000142   Section        2  libinit2.o(.ARM.Collect$$libinit$$0000002F)
    .ARM.Collect$$libshutdown$$00000000      0x10000144   Section        2  libshutdown.o(.ARM.Collect$$libshutdown$$00000000)
    .ARM.Collect$$libshutdown$$00000003      0x10000146   Section        0  libshutdown2.o(.ARM.Collect$$libshutdown$$00000003)
    .ARM.Collect$$libshutdown$$00000006      0x10000146   Section        0  libshutdown2.o(.ARM.Collect$$libshutdown$$00000006)
    .ARM.Collect$$libshutdown$$00000009      0x10000146   Section        0  libshutdown2.o(.ARM.Collect$$libshutdown$$00000009)
    .ARM.Collect$$libshutdown$$0000000B      0x10000146   Section        0  libshutdown2.o(.ARM.Collect$$libshutdown$$0000000B)
    .ARM.Collect$$libshutdown$$0000000E      0x10000146   Section        0  libshutdown2.o(.ARM.Collect$$libshutdown$$0000000E)
    .ARM.Collect$$libshutdown$$0000000F      0x10000146   Section        2  libshutdown2.o(.ARM.Collect$$libshutdown$$0000000F)
    .ARM.Collect$$rtentry$$00000000          0x10000148   Section        0  rtentry.o(.ARM.Collect$$rtentry$$00000000)
    .ARM.Collect$$rtentry$$00000002          0x10000148   Section        0  rtentry2.o(.ARM.Collect$$rtentry$$00000002)
    .ARM.Collect$$rtentry$$00000004          0x10000148   Section        6  rtentry4.o(.ARM.Collect$$rtentry$$00000004)
    .ARM.Collect$$rtentry$$00000009          0x1000014e   Section        0  rtentry2.o(.ARM.Collect$$rtentry$$00000009)
    .ARM.Collect$$rtentry$$0000000A          0x1000014e   Section        4  rtentry2.o(.ARM.Collect$$rtentry$$0000000A)
    .ARM.Collect$$rtentry$$0000000C          0x10000152   Section        0  rtentry2.o(.ARM.Collect$$rtentry$$0000000C)
    .ARM.Collect$$rtentry$$0000000D          0x10000152   Section        8  rtentry2.o(.ARM.Collect$$rtentry$$0000000D)
    .ARM.Collect$$rtexit$$00000000           0x1000015a   Section        2  rtexit.o(.ARM.Collect$$rtexit$$00000000)
    .ARM.Collect$$rtexit$$00000002           0x1000015c   Section        0  rtexit2.o(.ARM.Collect$$rtexit$$00000002)
    .ARM.Collect$$rtexit$$00000003           0x1000015c   Section        4  rtexit2.o(.ARM.Collect$$rtexit$$00000003)
    .ARM.Collect$$rtexit$$00000004           0x10000160   Section        6  rtexit2.o(.ARM.Collect$$rtexit$$00000004)
    .emb_text                                0x10000168   Section       56  rt_memcpy.o(.emb_text)
    .text                                    0x100001a0   Section        0  system_xn11lxxx.o(.text)
    .text                                    0x10000220   Section       48  startup_xn11lxxx.o(.text)
    .text                                    0x10000250   Section        0  xn_uart.o(.text)
    NVIC_DisableIRQ                          0x100004c7   Thumb Code    14  xn_uart.o(.text)
    .text                                    0x1000050c   Section        0  main.o(.text)
    .text                                    0x10000580   Section      346  aeabi_sdiv.o(.text)
    .text                                    0x100006da   Section        0  heapauxi.o(.text)
    .text                                    0x100006e0   Section       62  sys_stackheap_outer.o(.text)
    .text                                    0x1000071e   Section        0  exit.o(.text)
    .text                                    0x1000072c   Section        8  libspace.o(.text)
    .text                                    0x10000734   Section        0  sys_exit.o(.text)
    .text                                    0x10000740   Section        2  use_no_semi.o(.text)
    .text                                    0x10000742   Section        0  indicate_semi.o(.text)
    .constdata                               0x10000744   Section       64  system_xn11lxxx.o(.constdata)
    .data                                    0x10001000   Section        8  system_xn11lxxx.o(.data)
    .data                                    0x10001008   Section       16  xn_uart.o(.data)
    .bss                                     0x10001018   Section       64  xn_uart.o(.bss)
    .bss                                     0x10001058   Section       96  libspace.o(.bss)
    HEAP                                     0x100010b8   Section      256  startup_xn11lxxx.o(HEAP)
    Heap_Mem                                 0x100010b8   Data         256  startup_xn11lxxx.o(HEAP)
    STACK                                    0x100011b8   Section      512  startup_xn11lxxx.o(STACK)
    Stack_Mem                                0x100011b8   Data         512  startup_xn11lxxx.o(STACK)
    __initial_sp                             0x100013b8   Data           0  startup_xn11lxxx.o(STACK)

    Global Symbols

    Symbol Name                              Value     Ov Type        Size  Object(Section)

    BuildAttributes$$THM_ISAv3M$S$PE$A:L22$X:L11$S22$IEEE1$IW$USESV6$~STKCKD$USESV7$~SHL$OSPACE$ROPI$EBA8$UX$STANDARDLIB$REQ8$PRES8$EABIv2 0x00000000   Number         0  anon$$obj.o ABSOLUTE
    __ARM_use_no_argv                        0x00000000   Number         0  main.o ABSOLUTE
    __ARM_exceptions_init                     - Undefined Weak Reference
    __alloca_initialize                       - Undefined Weak Reference
    __cpp_initialize__aeabi_                  - Undefined Weak Reference
    __cxa_finalize                            - Undefined Weak Reference
    __rt_locale                               - Undefined Weak Reference
    __sigvec_lookup                           - Undefined Weak Reference
    _atexit_init                              - Undefined Weak Reference
    _call_atexit_fns                          - Undefined Weak Reference
    _clock_init                               - Undefined Weak Reference
    _fp_trap_init                             - Undefined Weak Reference
    _fp_trap_shutdown                         - Undefined Weak Reference
    _get_lc_collate                           - Undefined Weak Reference
    _get_lc_ctype                             - Undefined Weak Reference
    _get_lc_monetary                          - Undefined Weak Reference
    _get_lc_numeric                           - Undefined Weak Reference
    _get_lc_time                              - Undefined Weak Reference
    _getenv_init                              - Undefined Weak Reference
    _handle_redirection                       - Undefined Weak Reference
    _init_alloc                               - Undefined Weak Reference
    _init_user_alloc                          - Undefined Weak Reference
    _initio                                   - Undefined Weak Reference
    _rand_init                                - Undefined Weak Reference
    _signal_finish                            - Undefined Weak Reference
    _signal_init                              - Undefined Weak Reference
    _terminate_alloc                          - Undefined Weak Reference
    _terminate_user_alloc                     - Undefined Weak Reference
    _terminateio                              - Undefined Weak Reference
    __Vectors_Size                           0x000000c0   Number         0  startup_xn11lxxx.o ABSOLUTE
    __Vectors                                0x10000000   Data           4  startup_xn11lxxx.o(RESET)
    __Vectors_End                            0x100000c0   Data           0  startup_xn11lxxx.o(RESET)
    __main                                   0x100000c1   Thumb Code     8  __main.o(!!!main)
    __scatterload                            0x100000c9   Thumb Code     0  __scatter.o(!!!scatter)
    __scatterload_rt2                        0x100000c9   Thumb Code    52  __scatter.o(!!!scatter)
    __scatterload_rt2_thumb_only             0x100000c9   Thumb Code     0  __scatter.o(!!!scatter)
    __scatterload_null                       0x100000d9   Thumb Code     0  __scatter.o(!!!scatter)
    __scatterload_copy                       0x10000105   Thumb Code    26  __scatter_copy.o(!!handler_copy)
    __scatterload_zeroinit                   0x10000121   Thumb Code    28  __scatter_zi.o(!!handler_zi)
    __rt_lib_init                            0x1000013d   Thumb Code     0  libinit.o(.ARM.Collect$$libinit$$00000000)
    __rt_lib_init_alloca_1                   0x10000143   Thumb Code     0  libinit2.o(.ARM.Collect$$libinit$$0000002A)
    __rt_lib_init_argv_1                     0x10000143   Thumb Code     0  libinit2.o(.ARM.Collect$$libinit$$00000028)
    __rt_lib_init_atexit_1                   0x10000143   Thumb Code     0  libinit2.o(.ARM.Collect$$libinit$$00000017)
    __rt_lib_init_clock_1                    0x10000143   Thumb Code     0  libinit2.o(.ARM.Collect$$libinit$$0000001D)
    __rt_lib_init_cpp_1                      0x10000143   Thumb Code     0  libinit2.o(.ARM.Collect$$libinit$$0000002E)
    __rt_lib_init_exceptions_1               0x10000143   Thumb Code     0  libinit2.o(.ARM.Collect$$libinit$$0000002C)
    __rt_lib_init_fp_trap_1                  0x10000143   Thumb Code     0  libinit2.o(.ARM.Collect$$libinit$$0000001B)
    __rt_lib_init_getenv_1                   0x10000143   Thumb Code     0  libinit2.o(.ARM.Collect$$libinit$$0000001F)
    __rt_lib_init_heap_1                     0x10000143   Thumb Code     0  libinit2.o(.ARM.Collect$$libinit$$00000006)
    __rt_lib_init_lc_collate_1               0x10000143   Thumb Code     0  libinit2.o(.ARM.Collect$$libinit$$0000000D)
    __rt_lib_init_lc_ctype_1                 0x10000143   Thumb Code     0  libinit2.o(.ARM.Collect$$libinit$$0000000F)
    __rt_lib_init_lc_monetary_1              0x10000143   Thumb Code     0  libinit2.o(.ARM.Collect$$libinit$$00000011)
    __rt_lib_init_lc_numeric_1               0x10000143   Thumb Code     0  libinit2.o(.ARM.Collect$$libinit$$00000013)
    __rt_lib_init_lc_time_1                  0x10000143   Thumb Code     0  libinit2.o(.ARM.Collect$$libinit$$00000015)
    __rt_lib_init_rand_1                     0x10000143   Thumb Code     0  libinit2.o(.ARM.Collect$$libinit$$0000000A)
    __rt_lib_init_return                     0x10000143   Thumb Code     0  libinit2.o(.ARM.Collect$$libinit$$0000002F)
    __rt_lib_init_signal_1                   0x10000143   Thumb Code     0  libinit2.o(.ARM.Collect$$libinit$$00000019)
    __rt_lib_init_stdio_1                    0x10000143   Thumb Code     0  libinit2.o(.ARM.Collect$$libinit$$00000021)
    __rt_lib_init_user_alloc_1               0x10000143   Thumb Code     0  libinit2.o(.ARM.Collect$$libinit$$00000008)
    __rt_lib_shutdown                        0x10000145   Thumb Code     0  libshutdown.o(.ARM.Collect$$libshutdown$$00000000)
    __rt_lib_shutdown_fp_trap_1              0x10000147   Thumb Code     0  libshutdown2.o(.ARM.Collect$$libshutdown$$00000006)
    __rt_lib_shutdown_heap_1                 0x10000147   Thumb Code     0  libshutdown2.o(.ARM.Collect$$libshutdown$$0000000E)
    __rt_lib_shutdown_return                 0x10000147   Thumb Code     0  libshutdown2.o(.ARM.Collect$$libshutdown$$0000000F)
    __rt_lib_shutdown_signal_1               0x10000147   Thumb Code     0  libshutdown2.o(.ARM.Collect$$libshutdown$$00000009)
    __rt_lib_shutdown_stdio_1                0x10000147   Thumb Code     0  libshutdown2.o(.ARM.Collect$$libshutdown$$00000003)
    __rt_lib_shutdown_user_alloc_1           0x10000147   Thumb Code     0  libshutdown2.o(.ARM.Collect$$libshutdown$$0000000B)
    __rt_entry                               0x10000149   Thumb Code     0  rtentry.o(.ARM.Collect$$rtentry$$00000000)
    __rt_entry_presh_1                       0x10000149   Thumb Code     0  rtentry2.o(.ARM.Collect$$rtentry$$00000002)
    __rt_entry_sh                            0x10000149   Thumb Code     0  rtentry4.o(.ARM.Collect$$rtentry$$00000004)
    __rt_entry_li                            0x1000014f   Thumb Code     0  rtentry2.o(.ARM.Collect$$rtentry$$0000000A)
    __rt_entry_postsh_1                      0x1000014f   Thumb Code     0  rtentry2.o(.ARM.Collect$$rtentry$$00000009)
    __rt_entry_main                          0x10000153   Thumb Code     0  rtentry2.o(.ARM.Collect$$rtentry$$0000000D)
    __rt_entry_postli_1                      0x10000153   Thumb Code     0  rtentry2.o(.ARM.Collect$$rtentry$$0000000C)
    __rt_exit                                0x1000015b   Thumb Code     0  rtexit.o(.ARM.Collect$$rtexit$$00000000)
    __rt_exit_ls                             0x1000015d   Thumb Code     0  rtexit2.o(.ARM.Collect$$rtexit$$00000003)
    __rt_exit_prels_1                        0x1000015d   Thumb Code     0  rtexit2.o(.ARM.Collect$$rtexit$$00000002)
    __rt_exit_exit                           0x10000161   Thumb Code     0  rtexit2.o(.ARM.Collect$$rtexit$$00000004)
    __aeabi_memcpy4                          0x10000169   Thumb Code    56  rt_memcpy.o(.emb_text)
    __aeabi_memcpy8                          0x10000169   Thumb Code     0  rt_memcpy.o(.emb_text)
    SystemCoreClockUpdate                    0x100001a1   Thumb Code   106  system_xn11lxxx.o(.text)
    SystemInit                               0x1000020b   Thumb Code     2  system_xn11lxxx.o(.text)
    Reset_Handler                            0x10000221   Thumb Code     4  startup_xn11lxxx.o(.text)
    NMI_Handler                              0x10000225   Thumb Code     2  startup_xn11lxxx.o(.text)
    HardFault_Handler                        0x10000227   Thumb Code     2  startup_xn11lxxx.o(.text)
    SVC_Handler                              0x10000229   Thumb Code     2  startup_xn11lxxx.o(.text)
    PendSV_Handler                           0x1000022b   Thumb Code     2  startup_xn11lxxx.o(.text)
    SysTick_Handler                          0x1000022d   Thumb Code     2  startup_xn11lxxx.o(.text)
    ADC_IRQHandler                           0x1000022f   Thumb Code     0  startup_xn11lxxx.o(.text)
    BOD_IRQHandler                           0x1000022f   Thumb Code     0  startup_xn11lxxx.o(.text)
    GPIO0_IRQHandler                         0x1000022f   Thumb Code     0  startup_xn11lxxx.o(.text)
    GPIO1_IRQHandler                         0x1000022f   Thumb Code     0  startup_xn11lxxx.o(.text)
    GPIO2_IRQHandler                         0x1000022f   Thumb Code     0  startup_xn11lxxx.o(.text)
    PWM_FAULT_IRQHandler                     0x1000022f   Thumb Code     0  startup_xn11lxxx.o(.text)
    PWM_TIMER_IRQHandler                     0x1000022f   Thumb Code     0  startup_xn11lxxx.o(.text)
    RTC_IRQHandler                           0x1000022f   Thumb Code     0  startup_xn11lxxx.o(.text)
    SPI_IRQHandler                           0x1000022f   Thumb Code     0  startup_xn11lxxx.o(.text)
    TIMER16_0_IRQHandler                     0x1000022f   Thumb Code     0  startup_xn11lxxx.o(.text)
    TIMER16_1_IRQHandler                     0x1000022f   Thumb Code     0  startup_xn11lxxx.o(.text)
    TIMER16_2_IRQHandler                     0x1000022f   Thumb Code     0  startup_xn11lxxx.o(.text)
    TIMER16_3_IRQHandler                     0x1000022f   Thumb Code     0  startup_xn11lxxx.o(.text)
    TWS_IRQHandler                           0x1000022f   Thumb Code     0  startup_xn11lxxx.o(.text)
    UART1_IRQHandler                         0x1000022f   Thumb Code     0  startup_xn11lxxx.o(.text)
    WAKEUP_IRQHandler                        0x1000022f   Thumb Code     0  startup_xn11lxxx.o(.text)
    WDT_IRQHandler                           0x1000022f   Thumb Code     0  startup_xn11lxxx.o(.text)
    __user_initial_stackheap                 0x10000231   Thumb Code     0  startup_xn11lxxx.o(.text)
    UART0AutoDetect                          0x10000251   Thumb Code    78  xn_uart.o(.text)
    SetUART0Pin                              0x1000029f   Thumb Code    10  xn_uart.o(.text)
    UART0Init                                0x100002a9   Thumb Code    66  xn_uart.o(.text)
    UART0INTSet                              0x100002eb   Thumb Code    46  xn_uart.o(.text)
    UART0_IRQHandler                         0x10000319   Thumb Code   220  xn_uart.o(.text)
    UART0Send                                0x100003f5   Thumb Code    58  xn_uart.o(.text)
    UART0PutStr                              0x1000042f   Thumb Code    56  xn_uart.o(.text)
    UART0PutHex                              0x10000467   Thumb Code    52  xn_uart.o(.text)
    UART0GetChar                             0x1000049b   Thumb Code    44  xn_uart.o(.text)
    main                                     0x1000050d   Thumb Code    78  main.o(.text)
    __aeabi_uidiv                            0x10000581   Thumb Code     0  aeabi_sdiv.o(.text)
    __aeabi_uidivmod                         0x10000581   Thumb Code    20  aeabi_sdiv.o(.text)
    __aeabi_idiv                             0x10000595   Thumb Code     0  aeabi_sdiv.o(.text)
    __aeabi_idivmod                          0x10000595   Thumb Code   326  aeabi_sdiv.o(.text)
    __use_two_region_memory                  0x100006db   Thumb Code     2  heapauxi.o(.text)
    __rt_heap_escrow$2region                 0x100006dd   Thumb Code     2  heapauxi.o(.text)
    __rt_heap_expand$2region                 0x100006df   Thumb Code     2  heapauxi.o(.text)
    __user_setup_stackheap                   0x100006e1   Thumb Code    62  sys_stackheap_outer.o(.text)
    exit                                     0x1000071f   Thumb Code    12  exit.o(.text)
    __user_libspace                          0x1000072d   Thumb Code     8  libspace.o(.text)
    __user_perproc_libspace                  0x1000072d   Thumb Code     0  libspace.o(.text)
    __user_perthread_libspace                0x1000072d   Thumb Code     0  libspace.o(.text)
    _sys_exit                                0x10000735   Thumb Code     8  sys_exit.o(.text)
    __I$use$semihosting                      0x10000741   Thumb Code     0  use_no_semi.o(.text)
    __use_no_semihosting_swi                 0x10000741   Thumb Code     2  use_no_semi.o(.text)
    __semihosting_library_function           0x10000743   Thumb Code     0  indicate_semi.o(.text)
    Region$$Table$$Base                      0x10000784   Number         0  anon$$obj.o(Region$$Table)
    Region$$Table$$Limit                     0x100007a4   Number         0  anon$$obj.o(Region$$Table)
    SystemCoreClock                          0x10001000   Data           4  system_xn11lxxx.o(.data)
    MainClock                                0x10001004   Data           4  system_xn11lxxx.o(.data)
    UART0Head                                0x10001008   Data           4  xn_uart.o(.data)
    UART0Tail                                0x1000100c   Data           4  xn_uart.o(.data)
    UART0SendNo                              0x10001010   Data           4  xn_uart.o(.data)
    UART0SendPtr                             0x10001014   Data           4  xn_uart.o(.data)
    UART0Buffer                              0x10001018   Data          64  xn_uart.o(.bss)
    __libspace_start                         0x10001058   Data          96  libspace.o(.bss)
    __temporary_stack_top$libspace           0x100010b8   Data           0  libspace.o(.bss)



==============================================================================

Memory Map of the image

  Image Entry point : 0x100000c1

  Load Region LR_IROM1 (Base: 0x10000000, Size: 0x000007bc, Max: 0x00001000, ABSOLUTE)

    Execution Region ER_IROM1 (Base: 0x10000000, Size: 0x000007a4, Max: 0x00001000, ABSOLUTE)

    Base Addr    Size         Type   Attr      Idx    E Section Name        Object

    0x10000000   0x000000c0   Data   RO           50    RESET               startup_xn11lxxx.o
    0x100000c0   0x00000008   Code   RO          113  * !!!main             c_p.l(__main.o)
    0x100000c8   0x0000003c   Code   RO          283    !!!scatter          c_p.l(__scatter.o)
    0x10000104   0x0000001a   Code   RO          285    !!handler_copy      c_p.l(__scatter_copy.o)
    0x1000011e   0x00000002   PAD
    0x10000120   0x0000001c   Code   RO          287    !!handler_zi        c_p.l(__scatter_zi.o)
    0x1000013c   0x00000006   Code   RO          156    .ARM.Collect$$libinit$$00000000  c_p.l(libinit.o)
    0x10000142   0x00000000   Code   RO          171    .ARM.Collect$$libinit$$00000006  c_p.l(libinit2.o)
    0x10000142   0x00000000   Code   RO          173    .ARM.Collect$$libinit$$00000008  c_p.l(libinit2.o)
    0x10000142   0x00000000   Code   RO          175    .ARM.Collect$$libinit$$0000000A  c_p.l(libinit2.o)
    0x10000142   0x00000000   Code   RO          178    .ARM.Collect$$libinit$$0000000D  c_p.l(libinit2.o)
    0x10000142   0x00000000   Code   RO          180    .ARM.Collect$$libinit$$0000000F  c_p.l(libinit2.o)
    0x10000142   0x00000000   Code   RO          182    .ARM.Collect$$libinit$$00000011  c_p.l(libinit2.o)
    0x10000142   0x00000000   Code   RO          184    .ARM.Collect$$libinit$$00000013  c_p.l(libinit2.o)
    0x10000142   0x00000000   Code   RO          186    .ARM.Collect$$libinit$$00000015  c_p.l(libinit2.o)
    0x10000142   0x00000000   Code   RO          188    .ARM.Collect$$libinit$$00000017  c_p.l(libinit2.o)
    0x10000142   0x00000000   Code   RO          190    .ARM.Collect$$libinit$$00000019  c_p.l(libinit2.o)
    0x10000142   0x00000000   Code   RO          192    .ARM.Collect$$libinit$$0000001B  c_p.l(libinit2.o)
    0x10000142   0x00000000   Code   RO          194    .ARM.Collect$$libinit$$0000001D  c_p.l(libinit2.o)
    0x10000142   0x00000000   Code   RO          196    .ARM.Collect$$libinit$$0000001F  c_p.l(libinit2.o)
    0x10000142   0x00000000   Code   RO          198    .ARM.Collect$$libinit$$00000021  c_p.l(libinit2.o)
    0x10000142   0x00000000   Code   RO          202    .ARM.Collect$$libinit$$00000028  c_p.l(libinit2.o)
    0x10000142   0x00000000   Code   RO          204    .ARM.Collect$$libinit$$0000002A  c_p.l(libinit2.o)
    0x10000142   0x00000000   Code   RO          206    .ARM.Collect$$libinit$$0000002C  c_p.l(libinit2.o)
    0x10000142   0x00000000   Code   RO          208    .ARM.Collect$$libinit$$0000002E  c_p.l(libinit2.o)
    0x10000142   0x00000002   Code   RO          209    .ARM.Collect$$libinit$$0000002F  c_p.l(libinit2.o)
    0x10000144   0x00000002   Code   RO          241    .ARM.Collect$$libshutdown$$00000000  c_p.l(libshutdown.o)
    0x10000146   0x00000000   Code   RO          268    .ARM.Collect$$libshutdown$$00000003  c_p.l(libshutdown2.o)
    0x10000146   0x00000000   Code   RO          271    .ARM.Collect$$libshutdown$$00000006  c_p.l(libshutdown2.o)
    0x10000146   0x00000000   Code   RO          274    .ARM.Collect$$libshutdown$$00000009  c_p.l(libshutdown2.o)
    0x10000146   0x00000000   Code   RO          276    .ARM.Collect$$libshutdown$$0000000B  c_p.l(libshutdown2.o)
    0x10000146   0x00000000   Code   RO          279    .ARM.Collect$$libshutdown$$0000000E  c_p.l(libshutdown2.o)
    0x10000146   0x00000002   Code   RO          280    .ARM.Collect$$libshutdown$$0000000F  c_p.l(libshutdown2.o)
    0x10000148   0x00000000   Code   RO          115    .ARM.Collect$$rtentry$$00000000  c_p.l(rtentry.o)
    0x10000148   0x00000000   Code   RO          122    .ARM.Collect$$rtentry$$00000002  c_p.l(rtentry2.o)
    0x10000148   0x00000006   Code   RO          137    .ARM.Collect$$rtentry$$00000004  c_p.l(rtentry4.o)
    0x1000014e   0x00000000   Code   RO          124    .ARM.Collect$$rtentry$$00000009  c_p.l(rtentry2.o)
    0x1000014e   0x00000004   Code   RO          125    .ARM.Collect$$rtentry$$0000000A  c_p.l(rtentry2.o)
    0x10000152   0x00000000   Code   RO          127    .ARM.Collect$$rtentry$$0000000C  c_p.l(rtentry2.o)
    0x10000152   0x00000008   Code   RO          128    .ARM.Collect$$rtentry$$0000000D  c_p.l(rtentry2.o)
    0x1000015a   0x00000002   Code   RO          161    .ARM.Collect$$rtexit$$00000000  c_p.l(rtexit.o)
    0x1000015c   0x00000000   Code   RO          215    .ARM.Collect$$rtexit$$00000002  c_p.l(rtexit2.o)
    0x1000015c   0x00000004   Code   RO          216    .ARM.Collect$$rtexit$$00000003  c_p.l(rtexit2.o)
    0x10000160   0x00000006   Code   RO          217    .ARM.Collect$$rtexit$$00000004  c_p.l(rtexit2.o)
    0x10000166   0x00000002   PAD
    0x10000168   0x00000038   Code   RO          103    .emb_text           c_p.l(rt_memcpy.o)
    0x100001a0   0x00000080   Code   RO           13    .text               system_xn11lxxx.o
    0x10000220   0x00000030   Code   RO           51    .text               startup_xn11lxxx.o
    0x10000250   0x000002bc   Code   RO           56    .text               xn_uart.o
    0x1000050c   0x00000074   Code   RO           86    .text               main.o
    0x10000580   0x0000015a   Code   RO          107    .text               c_p.l(aeabi_sdiv.o)
    0x100006da   0x00000006   Code   RO          111    .text               c_p.l(heapauxi.o)
    0x100006e0   0x0000003e   Code   RO          141    .text               c_p.l(sys_stackheap_outer.o)
    0x1000071e   0x0000000c   Code   RO          144    .text               c_p.l(exit.o)
    0x1000072a   0x00000002   PAD
    0x1000072c   0x00000008   Code   RO          157    .text               c_p.l(libspace.o)
    0x10000734   0x0000000c   Code   RO          212    .text               c_p.l(sys_exit.o)
    0x10000740   0x00000002   Code   RO          230    .text               c_p.l(use_no_semi.o)
    0x10000742   0x00000000   Code   RO          232    .text               c_p.l(indicate_semi.o)
    0x10000742   0x00000002   PAD
    0x10000744   0x00000040   Data   RO           14    .constdata          system_xn11lxxx.o
    0x10000784   0x00000020   Data   RO          281    Region$$Table       anon$$obj.o


    Execution Region RW_IRAM1 (Base: 0x10001000, Size: 0x000003b8, Max: 0x00001000, ABSOLUTE)

    Base Addr    Size         Type   Attr      Idx    E Section Name        Object

    0x10001000   0x00000008   Data   RW           15    .data               system_xn11lxxx.o
    0x10001008   0x00000010   Data   RW           58    .data               xn_uart.o
    0x10001018   0x00000040   Zero   RW           57    .bss                xn_uart.o
    0x10001058   0x00000060   Zero   RW          158    .bss                c_p.l(libspace.o)
    0x100010b8   0x00000100   Zero   RW           49    HEAP                startup_xn11lxxx.o
    0x100011b8   0x00000200   Zero   RW           48    STACK               startup_xn11lxxx.o


==============================================================================

Image component sizes


      Code (inc. data)   RO Data    RW Data    ZI Data      Debug   Object Name

         0          0          0          0          0       4156   core_cm0.o
       116         38          0          0          0        407   main.o
        48         22        192          0        768        640   startup_xn11lxxx.o
       128         20         64          8          0       8307   system_xn11lxxx.o
       700         56          0         16         64       8447   xn_uart.o

    ----------------------------------------------------------------------
       992        136        288         24        832      21957   Object Totals
         0          0         32          0          0          0   (incl. Generated)
         0          0          0          0          0          0   (incl. Padding)

    ----------------------------------------------------------------------

      Code (inc. data)   RO Data    RW Data    ZI Data      Debug   Library Member Name

         8          0          0          0          0         68   __main.o
        60          8          0          0          0          0   __scatter.o
        26          0          0          0          0          0   __scatter_copy.o
        28          0          0          0          0          0   __scatter_zi.o
       346          0          0          0          0         92   aeabi_sdiv.o
        12          0          0          0          0         64   exit.o
         6          0          0          0          0        136   heapauxi.o
         0          0          0          0          0          0   indicate_semi.o
         6          0          0          0          0          0   libinit.o
         2          0          0          0          0          0   libinit2.o
         2          0          0          0          0          0   libshutdown.o
         2          0          0          0          0          0   libshutdown2.o
         8          4          0          0         96         68   libspace.o
        56          0          0          0          0         68   rt_memcpy.o
         0          0          0          0          0          0   rtentry.o
        12          0          0          0          0          0   rtentry2.o
         6          0          0          0          0          0   rtentry4.o
         2          0          0          0          0          0   rtexit.o
        10          0          0          0          0          0   rtexit2.o
        12          4          0          0          0         60   sys_exit.o
        62          0          0          0          0         80   sys_stackheap_outer.o
         2          0          0          0          0         68   use_no_semi.o

    ----------------------------------------------------------------------
       676         16          0          0         96        704   Library Totals
         8          0          0          0          0          0   (incl. Padding)

    ----------------------------------------------------------------------

      Code (inc. data)   RO Data    RW Data    ZI Data      Debug   Library Name

       668         16          0          0         96        704   c_p.l

    ----------------------------------------------------------------------
       676         16          0          0         96        704   Library Totals

    ----------------------------------------------------------------------

==============================================================================


      Code (inc. data)   RO Data    RW Data    ZI Data      Debug   

      1668        152        288         24        928      22129   Grand Totals
      1668        152        288         24        928      22129   ELF Image Totals
      1668        152        288         24          0          0   ROM Totals

==============================================================================

    Total RO  Size (Code + RO Data)                 1956 (   1.91kB)
    Total RW  Size (RW Data + ZI Data)               952 (   0.93kB)
    Total ROM Size (Code + RO Data + RW Data)       1980 (   1.93kB)

==============================================================================

